:020000040100F9
:10000000FD62938202400100FD12E39E02FE374131
:10001000000213010100B701000293810100B7152E
:100020000001938505003716000113060603B70685
:1000300000029386060039A083A2050023A0560083
:1000400091059106E3EAC5FEB71500019385050306
:100050003716000113060603B7060002938606262C
:1000600039A083A2050023A0560091059106E3EA7A
:10007000C5FEB70500029385050337060002130687
:10008000062621A023A005009105E3EDC5FEB700DB
:100090000001E780C00AB7000001E780C00AB7107E
:1000A0000001E780808473005010F5BF828000005B
:1000B0000000000000000000000000000000000040
:1000C0006F004000197106C20AC40EC612C816CAD3
:1000D0001ACC1ECE22D026D22AD42ED632D836DA48
:1000E0003ADC3EDEC2C0C6C2CAC4CEC6D2C8D6CA78
:1000F000DACCDECEE2D0E6D2EAD4EED6F2D8F6DA28
:10010000FADCFEDE970000009380E00482909240CB
:100110002241B2414242D2426243F24302549254DB
:100120002255B2554256D2566257F2570648964863
:100130002649B649464AD64A664BF64B065C965C5B
:10014000265DB65D465ED65E665FF65F096173004A
:10015000203001A03D432A876373C3029377F700E1
:10016000BDEFADE5937606FF3D8ABA960CC34CC34E
:100170000CC74CC74107E36BD7FE11E28280B30680
:10018000C3408A069702000096966780A600230760
:10019000B700A306B7002306B700A305B7002305E1
:1001A000B700A304B7002304B700A303B7002303D9
:1001B000B700A302B7002302B700A301B7002301D1
:1001C000B700A300B7002300B700828093F5F50FB6
:1001D00093968500D58D93960501D58D61B793963D
:1001E00027009702000096968682E78086FA96801E
:1001F000C1171D8F3E96E374C3F8A5B7B707050076
:100200000947D8CFB7170500938707C0984385667D
:1002100093860640558F98C398471367074098C741
:10022000B71708009387074023A0070023A2070001
:1002300023A407001307B010D8C77D57D8CF354780
:1002400098C3D84F935657018D8AE5DE8280B71741
:1002500008009387074023A0070023A2070023A4D8
:10026000070023A607007D57D8CF23A40702B7179E
:100270000500938707C09843F1769386F63F758F04
:1002800098C398471377F7BF98C7B7070500094782
:1002900098D38280B71708009387074088D7D84F34
:1002A000137707046DDF82803707000203234704BA
:1002B000B706000237150800B7450F0023A406044F
:1002C0008147014613050540938515240328C50180
:1002D000B308F30013780802630C080205C2232256
:1002E000170537470F0023A4F60413070724639765
:1002F000E700B707000205472383E700B7170800A8
:1003000093870740C85342054181828005467DBFDF
:100310008507E39DB7FE7DD2B7470F00938707247B
:1003200023A4F60423221705E9B7411106C622C407
:1003300026C2AA84EF003024E1689388086A014845
:100340008147014781460146B70520C72685379476
:100350009800EF00B007130414687D1419E40D45EC
:10036000B240224492444101828085452685EF00B7
:10037000F02105897DF10145E5B7411122C437041B
:100380000002930704008C43B70700804AC0BE9563
:10039000B707000223AEB70206C626C293974501EF
:1003A000130404003709000289E713058900EF00F0
:1003B000102B0C40B70400029386C40413060010EF
:1003C00013058900EF00F0241C4037070002835614
:1003D0008703938707101CC013060010B68763F4C9
:1003E000C600930700101384C4041305F400938718
:1003F00007F01306100F814513040410231CF702A5
:10040000913BA2851385C4043D46EF00902923202B
:1004100004002322040023240400231604002307DD
:100420000400B240224492440249410182805D713D
:10043000130680028145280886C6293BBD47230C48
:10044000F1008947230EF1003ED2E1779387070838
:100450002C080A85231AF102F52BB64061618280CF
:100460005D71A2C4370400021305840086C6A6C2CB
:10047000CAC0C12513058400EF00007F8545130520
:100480008400EF00B0108D47814463E3A700AA8485
:10049000894513058400EF00700F937725002A86A5
:1004A00089E7136625001376F60FA68513058400E9
:1004B000EF003011E1689388086A014881470147DD
:1004C00081460146B7052038130584000127E168FD
:1004D00038009388086A1308000285468147014660
:1004E000B70599EB1305840023040100C525B71552
:1004F00000015146938585FE6800EF00901A1309AC
:100500008400832709006C0051463ED085473ED2C7
:100510006810C1673ED4EF00D018B70607009C42B0
:100520003707F1FF7D17F98F08109CC2A925B64047
:1005300026449644064961618280411106C6013B0A
:100540000537B707008073905730B700008082905E
:10055000B2404101828041113707000222C406C621
:100560009307070083C76700854613040700638E5F
:10057000D70009476388E70023030400B240224400
:10058000410182801305000F3133B71708009387AC
:100590000740D84F218B09C7D84F13678700D8CFA2
:1005A000693FD9BF411106C622C426C24AC083474B
:1005B000350005476383E70811472A846389E7000C
:1005C0008DCFB24022449244024941018280B70754
:1005D000000283D7870391C34D3383474400034709
:1005E0005400E2074207BA97370700022320F704B6
:1005F000370700022320F700E9B7370900028354C8
:1006000089030346050093054500370500021305DD
:10061000C5042695EF00F00883470400BE94C20489
:10062000C180231C99029307F00FE3FC97F8224442
:10063000B24092440249410189B33D45A139B7070F
:10064000000283D7870391C30D3B2244B2409244FA
:1006500002494101DDB53707000241119306070049
:1006600003DF460026C4B704000283A2840422C626
:100670003715080037040002B7480F0037430F0052
:10068000370E00024AC28147232A04021309FFFFE2
:10069000814E814681458143014801461307070089
:1006A000130505409388182413030324130ECE1555
:1006B000636FE60363850E0009462303C70089C6FE
:1006C000B7060002A388F60299C1232A74026304C4
:1006D000080023A4540483476700A9E73244A244D6
:1006E0001249370500021305C515410165BD814258
:1006F0000328C50113780802631B08028502E399E9
:1007000012FF89C6B7060002A388F60299C1232A00
:100710007402B7470F009387072423A4F404854786
:100720002303F7003244A244124941018280E38A44
:1007300062FC03284502937FF80F637D260113783E
:10074000F80FC29385453308CE002300F801050653
:100750000548B9BFB307704093F7F70F6394FF00E4
:100760008546D5B7854EEDBF011122CC4EC652C489
:1007700037040002B7490F00371ADCBA26CA4AC844
:1007800056C25AC006CE13040400370900029389EA
:10079000F923930A0003B7040002391A370B000249
:1007A000213683274904A303A40063F3F9007133BE
:1007B0008347640099C34533E5B783467400638873
:1007C0005605930700066381F60603C704038D47A9
:1007D000998F8E07B357FA0093F7F70F6393F606D6
:1007E0009307170093F7F70F2388F4021147639DCF
:1007F000E7003D45453413058B00053E29C113052F
:10080000000F493C238804022322090451BF3D45BF
:100810002322090423880402B53C793405052312F8
:10082000A4003D45853CADBF3D45232209042388F6
:1008300004028D340D3583476400B5FFDDB73D45B7
:10084000C9B723880402A9BF011106CE22CCC53640
:100850003704000213058400E92C130584002921C4
:10086000E1689388086A0148814778008546014617
:10087000B705D9EB1305840023060100812EE1683A
:100880009388086A01488147014781460146B705B8
:1008900038FF130584001D2E9532F9350547AA87C8
:1008A0006305E50209476300E506054591EBB706D8
:1008B0000600DC4A7D771307F73FF98FDCCA014554
:1008C00082807D1719EB0D4582809306004037A783
:1008D000070013070712B7050500905D7D8E75D2DE
:1008E000370606005C4A7D771307F73FF98FD58FEF
:1008F00041115CCA02C613073006B2476359F700BC
:10090000014541018280856693860680C9B7B2475A
:1009100085073EC6DDB791476307F50263EAA70086
:100920008547630AF50489476309F5040545828014
:10093000A147E31DF5FE0947094501A8FD1781EF11
:10094000C8D20D45828005470D45B7A7070093879C
:100950000712B7060500905E798E6DD28A05C98DA3
:100960004111CCD202C613073006B247635AF700D2
:100970000145410182801147C9BF21470145F1B7B7
:10098000B24785073EC6D5B70547AA876305E50286
:1009900009476304E506054591EBB70606009C4A46
:1009A0007D771307F73FF98F9CCA014582807D1739
:1009B00019EB0D4582809306004037A70700130707
:1009C0000712B7050500905D7D8E75D237070600CA
:1009D0001C4B7D761306F63FF18FD58F1CCB232C55
:1009E000070085471CCF411102C613073006B247E6
:1009F0006359F70001454101828085669386068030
:100A00006DBFB24785073EC6DDB711C98547630D87
:100A1000F50205458280FD1791EB0D458280094660
:100A2000B7A7070093870712B7060500985E718F76
:100A30007DD34111C8D602C613073006B2476357AB
:100A4000F7000145410182800546D9BFB2478507BD
:100A50003EC6EDB7011126CAB7040600DC4806CE33
:100A600022CC4AC84EC652C456C2F19BDCC89C4830
:100A70002A89C845F19B9CC8D84883C7C5012E84E4
:100A8000137737C08A07D98FDCC883C7D501984848
:100A90009A071377F7C393F7073CD98F9CC8FD3BA0
:100AA0000C44AA8A03454400BD351848B707050021
:100AB0002A8A98C358480850D8C3184C98C7E935B3
:100AC000AA8948509937834704002A8793F617006C
:100AD00089E6D44893E62600D4C893F6270099E621
:100AE00037060600544A93E6160054CA93F64700A8
:100AF00099E637060600144A93E6260014CAA18B2D
:100B000099E7B70606009C4A93E717009CCAF24093
:100B10006244232059012322490123243901232639
:100B2000E900D244B249224A924A4A8542490561C3
:100B30008280011106CE22CC02C402C62147B7072B
:100B4000050037550800D8C705448D478A85130529
:100B500005803EC022C2292A375508009307C003EA
:100B60008A851305058022C222C43EC01122F240AC
:100B7000624405618280411122C406C62A84553F21
:100B800018405C4F93E707015CCF1C441CCB5C40D2
:100B900085CB1C43B7061000D58F1CC3144C5C4892
:100BA000B240D606CE07D58F83460401C206D58F44
:100BB0008346C4012244E206D58F1CCF41018280C6
:100BC0001C43B706F0FFFD16F58FC1BF03230500D8
:100BD0002A8E0325C30113650502232EA3002324B7
:100BE000C3001396260149824D8E2326030123223A
:100BF000C300139605016354060299C20545B1CBA3
:100C000001476346D700639C08020D458280338606
:100C1000E700034606000507230AC300DDB799C2B3
:100C2000054505CB8147E3D0D7FE03260E000345DB
:100C300046013306F70085072300A600EDB783279A
:100C40000E00FD18DC4F93F70702D5DF11656D8D9F
:100C500011E18280B707070083C7470113F58500BC
:100C60001D8D3335A00082801C414147D8CF828042
:100C7000B7470800938707402A886304F508B757E9
:100C80000800938707806304F50A37470800630D5F
:100C9000E50A05458280331E1F013376DE0129C631
:100CA00083A3450088431393180033966F001346BF
:100CB000F6FF13F43300718D33146400418D88C343
:100CC000638B5302638C0302084303AEC500718D2E
:100CD000331E6E003365C50108C38842698E88459E
:100CE00033156500498E90C2850833D51E0145F540
:100CF0003244410182802326C801F9B72324C80168
:100D0000E1B7B716050037170500B717050093863A
:100D100046C1130707C19387C7C083AE050081484A
:100D2000054F8D4F914233D51E0105ED8280B716D8
:100D3000050037170500B7170500938606C213078D
:100D4000C7C1938787C1D1BFB71605003717050004
:100D5000B7170500938686C0130747C0938707C05F
:100D60006DBF331E1F013376DE0119E2850865BFB2
:100D7000411122C635B7E1689388086A0148814766
:100D8000014781460146B705200689B5011106CE07
:100D9000A307010089476393F502B7052035E16891
:100DA0001307F1009388086A014881478546014688
:100DB000313DF2400345F10005618280B705200511
:100DC000F9BF011106CE22CC26CA2306B100AA849F
:100DD000A306C1004D37E1689388086A01487C008A
:100DE000014789460146B785200126850964F93BFC
:100DF000130414717D1419E40D45F2406244D24489
:100E000005618280854526855137058965F501454F
:100E1000EDB7011106CE22CC26CA2E844AC8AA8478
:100E2000328936C6893FB247E16822869388086ACC
:100E300001480147CA86B7858002268561647933F7
:100E40001304146A7D1411C48545268581370589EC
:100E500075F9F2406244D244424905618280011131
:100E600006CE22CC26CA2EC6AA8431373246E16885
:100E70009388086A0148814701478146B705802069
:100E800026856164A1331304146A7D1411C4854559
:100E90002685ED3D058975F9F2406244D24405612D
:100EA0008280B3C7A5008D8BB308C500B1E78D471D
:100EB00063F4C704937735002A87B9EB13F6C8FFAC
:100EC000B306E6409307000263C8D706AE86BA872A
:100ED0006371C70203A806009107910623AE07FFBE
:100EE000E3EAC7FE9307F6FF998FF19B91073E97C0
:100EF000BE956366170182802A87637E150383C7C8
:100F0000050005078505A30FF7FEE39AE8FE82803A
:100F100083C60500050793773700A30FD7FE850525
:100F2000D1DF83C60500050793773700A30FD7FEEF
:100F30008505F9FF61B78280411122C613040002C2
:100F400083A3050083A2450083AF850003AFC500DE
:100F500083AE050103AE450103A3850103A8C501C6
:100F6000945113074702B307E640232E77FC232052
:100F700057FE2322F7FF2324E7FF2326D7FF23284A
:100F8000C7FF232A67FE232C07FF232ED7FE938556
:100F90004502E347F4FAAE86BA876371C70203A835
:100FA00006009107910623AE07FFE3EAC7FE930709
:100FB000F6FF998FF19B91073E97BE9563651701E8
:100FC00032444101828083C7050005078505A30FD0
:100FD000F7FEE387E8FE83C7050005078505A30F35
:100FE000F7FEE392E8FEE9BF2000000001000000E8
:100FF0000300000006000000EB00000000000000FD
:101000000000008000000000000007000000000059
:1010100000000000000000000000000000000000D0
:1010200000000000000000000000000000000000C0
:0400000501000000F6
:00000001FF
